:0400000000000000FC
:0400010000000000FB
:0400020000000000FA
:0400030000000000F9
:0400040000000000F8
:0400050001C60260CE
:04000600160400D705
:040007003A280D4046
:0400080000000000F4
:0400090000000000F3
:04000A000CC60360BD
:04000B001D04017758
:04000C003A280D4041
:04000D000FC6C0005A
:04000E0016200201B5
:04000F002EC60000F9
:040010003520020095
:0400110000000000EB
:0400120000000000EA
:0400130000000000E9
:0400140000000000E8
:0400150014C207E129
:040016003AC20700E3
:040017003B2000008A
:040018000ABE00001C
:040019003B20000088
:04001A0010C20720E9
:04001B003B20000086
:04001C000ABE000018
:04001D003B20000084
:04001E0031C20740A4
:04001F003B20000082
:040020000ABE000014
:040021003B20000080
:040022001BC2076096
:040023003B2000007E
:040024000ABE000010
:040025003B2000007C
:0400260016C2078077
:040027003B2000007A
:040028000ABE00000C
:040029003B20000078
:04002A003CC207A02D
:04002B003B20000076
:04002C000ABE000008
:04002D003B20000074
:04002E001DC207C028
:04002F003B20000072
:040030000ABE000004
:040031003B20000070
:0400320000000000CA
:04003300098A1621FF
:04003400320402C1CF
:0400350000000000C7
:0400360000000000C6
:0400370000000000C5
:0400380000000000C4
:0400390000000000C3
:04003A0000000000C2
:04003B002150000F41
:04003C0029C6180EAB
:04003D0027C601C110
:04003E00109017E91E
:04003F0019E600249A
:0400400033E600049F
:040041002A0408374E
:04004200343C40000A
:04004300098A1621EF
:040044003A0407E192
:0400450039E618255B
:0400460039E618255A
:040047000D0408F7A5
:04004800063C500022
:040049002FE6404519
:04004A000604095748
:04004B00063C50001F
:04004C0021040997EB
:04004D002BC602407C
:04004E003B280A043D
:04004F002E0409EF83
:0400500000000000AC
:00000001ff
